:020000040800F2
:10500000F8190020D5500008E577000875740008ED
:105010000000000000000000000000000000000090
:1050200000000000000000000000000035810008C2
:105030000000000000000000597F00081D820008E9
:10504000E7500008E7500008E7500008E750000864
:10505000E7500008795A0008E7500008E7500008B8
:1050600000000000E7500008B5590008E7500008AC
:10507000E7500008B575000800000000E750000880
:1050800000000000E75000080000000000000000E1
:10509000E750000800000000E7500008E750000853
:1050A000E7500008E7500008E75000086189000851
:1050B000E7500008E7500008000000000000000072
:1050C0000348854600F056FC004800470D9800084C
:1050D000F81900200448804704480047FEE7FEE72F
:1050E000FEE7FEE7FEE7FEE7B9820008C1500008D0
:1050F00030B50B46014600202022012409E00D4670
:10510000D5409D4205D31D469540491B25469540F7
:1051100040191546521E002DF1DC30BDF0B51FB40C
:105120000646002082B005464024019100901BE015
:10513000019922460F46304600F044FB049A059B35
:10514000801A994110D310461946224600F02AFBD6
:10515000361A8F410197224601200021009F00F05E
:1051600021FB38184D4100902046641E0028DFDCEA
:10517000019B00982946324607B0F0BD03460B4319
:105180009B0703D009E008C9121F08C0042AFAD2FD
:1051900003E00B780370401C491C521EF9D2704783
:1051A000D2B201E00270401C491EFBD270470022BF
:1051B000F6E710B513460A4604461946FFF7F0FF16
:1051C000204610BD30B504460020034600E05B1CBD
:1051D000934203D2E05CCD5C401BF8D030BDF8B503
:1051E00002464A40D40F42004B0052085B089A42E4
:1051F00002D20246084611464A0023D0C30D4A0097
:10520000DDB2120EAD1A202D35DA49020126490A07
:10521000F6058A19002C00D0524220214F1B11465E
:10522000B9402A411018C20D9A4221D0002C17D043
:10523000012D08DCDA05801AD20F8019D207DBB203
:1052400000F0ECFAF8BDDA05801A012340001B06D5
:10525000C01880185A428018CA0F1043490007E04E
:105260004908C2071143DA05801A801940088018DE
:1052700000F0CCFAF8BD61000122511A001BF7E7DB
:105280000122D2075140AAE70122D2075040A6E7E7
:1052900070B502464A40D50F40004A00ED0740086D
:1052A0005208002814D0002A12D0C40DD30D410298
:1052B0000120C0055202490A520AE41A09181218BC
:1052C0007D34914201D3641C00E04900002C01DAD6
:1052D000002070BD0023914201D3891A0343400886
:1052E00049000028F7D100290AD0914202D10121BA
:1052F000C90705E0914201D2012101E00121C94322
:10530000E005C018401900F081FA70BDF0B50746FD
:105310000846584087B0C00F049048000E46590018
:1053200040084908BC1A884105D2384631461E4615
:1053300017460B4602465800400810434CD0300D2B
:10534000039040055900400D490D0590401A029008
:10535000402872DA18030121000B09050843019067
:1053600004980092002805D00199524200208841FB
:1053700000920190029840210A1A0199009800F0C9
:1053800011FA05460C466B4607CB00F02CFAC01903
:105390007141039A0E0D0023D71756401A467A40E2
:1053A000164344D0049A002A2DD0029A012A039A67
:1053B00015DC1205C01A914101263605001C714109
:1053C000D20F059ED2070093019202962A462346E9
:1053D00000F06AFA07B0F0BD38463146FAE7160524
:1053E000224A0F46B218C01AB74101210905001C14
:1053F0004F4100187F41114618187941E20F1043C0
:105400006D19644113E0E2076D0815436408C20793
:105410001443039A01261205C01A91413605001C57
:105420007141CE07400830434908C01851412A460F
:10543000234600F02CFACDE7FFE704980122400054
:10544000C117121A00238B4104983146C417381A29
:10545000A141EEE730B40124E407634030BC55E7D6
:1054600030B40124E407614030BC4FE70000E0FFA6
:10547000F0B51FB488B00B990998002448400999E9
:10548000C00F490049080991C0070B9900904900D5
:1054900049080B9109990898A64608431CD00B9916
:1054A0000A98084318D0099801244000420D48008A
:1054B000410D099824050003000B204309900B9827
:1054C0000003000B20430B9050181C494018002289
:1054D00001901446104605E0002001460DB0F0BDD5
:1054E000032801DA034600E003239C46C11A0AAEF2
:1054F0000AE05F0008ADED5B4F00F75B7D430027DE
:10550000AA187C41491C5B1E6145F2DD410004ABD9
:105510005A522104120C0A43240C401C0828DFDBD9
:10552000019802900099704601910090059B049AA1
:105530000799069800F0B8F9D0E700000DFCFFFFCE
:10554000F0B50C465C4085B0E40FE40703944C00D2
:1055500000266408590094464908024602962243F0
:1055600021D062460A431ED06200570D4A000E0346
:105570002303550D012402462C492405781B1B0BDF
:10558000360B401823432643614600901C46501AB0
:10559000B44103D30098401C009002E09218009898
:1055A0005B41002803DA0020014605B0F0BD002071
:1055B000012109050746864611E064461D46141B75
:1055C000B54106D36546521BB341744607430C43AD
:1055D000A646CD0740084908284392185B41054676
:1055E0000D43EAD11046184313D060461946504087
:1055F0007140084306D06046101AB34106D201221A
:10560000002306E000220123DB0702E00122D2434F
:105610005310009874460105381C6141029C039D9B
:105620000019694100F033F9BFE70000FD030000F5
:10563000C217C10F504010B54018CA079623002169
:1056400000F0ECF810BD10B500229623114600F0D2
:10565000E5F810BD0EB5C217C10F5040CA0740187B
:105660000021054B0293019200910A460B4600F07F
:105670001BF903B000BD0000330400000EB505495E
:105680000291002100910A460B46019100F00CF9AD
:1056900003B000BD33040000410040020122400A73
:1056A000D205090E80187F2901DA0020704796295B
:1056B00003DC9622511AC8407047963988407047DB
:1056C00070B5CD0F4A0009030123090B1B051943CF
:1056D0000B4BED070024520D9A4201DA002070BDF9
:1056E000074B34339A4203DC9A1A00F06BF802E05D
:1056F0000449511888402C43F1D0404270BD00004D
:10570000FF030000CDFBFFFF4A0009030123090B43
:105710001B051943094B10B5520D9A4201DA0020BE
:1057200010BD064B34339A4203DC9A1A00F04AF853
:1057300010BD03495118884010BD0000FF03000050
:10574000CDFBFFFFC20FD207400040080BD0C10DB8
:105750000723DB01C91840020905400A1143C208AA
:10576000400711437047002001467047CB0FDB070D
:10577000490010B5490802460A4307D00A0D07241C
:105780000903E401090B121B002A01DC002010BDF3
:10579000C900440F0C43C100E018D205801800F086
:1057A00035F810BD10B5202A04DB0146203A91409F
:1057B000002010BD914020239C1A0346E34019436A
:1057C000904010BD10B5202A04DB0846203AD04096
:1057D000002110BD0B46D340D0402024A21A914096
:1057E0000843194610BD10B5202A06DBCB17084622
:1057F000203A1041C1170B4306E00B461341D0403D
:105800002024A21A91400843194610BD002904DA49
:10581000401C490001D140084000704770B400248A
:10582000050C05D11024000402D1002921D0112437
:10583000050E01D100020834050F01D10001241D1D
:10584000850F01D18000A41C002801DB4000641CEE
:10585000002908D020252E1B0D46F540A14000D080
:1058600001212943084301061B1B000ADB1D02D549
:10587000002070BC7047DB05181880180029F8DA82
:10588000401C4900F5D170BC40084000704710B57D
:10589000002B08DA0024401C614192185B411A4336
:1058A00001D14008400010BDF0B51FB482B00546DC
:1058B0000C0003D0084603F02BF902E003F028F9AE
:1058C00020300246009021462846FFF76BFF049BDC
:1058D000059A04460F4618431143084314D018464E
:1058E00010431BD0009840210A1A18460599FFF76B
:1058F00069FF05460E46009A05990498FFF752FF86
:10590000084305D0012004E02046394607B0F0BD29
:105910000020C11705430E432C43374300990E98CE
:105920006305401A7905E40A00220C43FD0A0A3097
:1059300002D500200146E9E70105101969410C9CD8
:105940000D9D00196941FFF7A2FFDFE710B500299F
:1059500004DB0124E40740428C412146002B04DB98
:105960001C460123DB075242A341994200D19042D9
:1059700010BD0000064C0125064E05E0E36807CC8B
:105980002B430C3C98471034B442F7D3FFF79CFBF1
:10599000009B0008209B000810B500231A4603E076
:1059A000845CE3189BB2521C8A42F9D3D84380B27C
:1059B00010BD000010B5034800F0DEFA024800F008
:1059C000DBFA10BD981500205015002030B5446C4E
:1059D0001C252C400125A540046C656004686360AB
:1059E0008368102B036803D099600068C26030BDE3
:1059F0009A600068C16030BD1049012048720220E1
:105A00005E31487203203C39487204200E394872D6
:105A10000A4B0B495A1C08785871497899712333FD
:105A200018715971203318775977107551751A46C6
:105A30001E32107551751076517670473411002062
:105A4000E000002010B502F04BFB202002F0DCFB50
:105A5000012003F00DFC002002F0D6FB044803F007
:105A6000ABFA044803F0A8FD002003F0DDFD10BDF3
:105A7000A00000208380000070B5052001210007F0
:105A800000F0B8FC00240D4D002800D02C6002214D
:105A90000B4800F0AFFC002808D10A482C600088B1
:105AA0000A2148430849088002F086FF012000F0DF
:105AB000D9FB022000F0D6FB70BD0000F8000020EA
:105AC00000040050C8000020D800002070470000EB
:105AD00010B5084900224A6107494B684C15234319
:105AE0004B604B68082423434B60C009C00102602F
:105AF00010BD0000E0150020002002407FB5002509
:105B00000C460646039500F07DFBE009029003A9D0
:105B100001960095684600F00DFB002804D000F0C7
:105B200045FB002004B070BD00F040FB0120F9E708
:105B300010B5002302E0C45CCC545B1C9342FAD342
:105B400010BD000010B5214A00219069C30520480E
:105B500004D54169022319434161911593699B055D
:105B600005D54369012423434361630219439369C3
:105B70005B0505D54369082423434361E3011943C9
:105B800093691B0505D543690424234343616302DC
:105B9000194393699B0405D543691024234343614A
:105BA0006302194393699B0304D5446920231C4372
:105BB000446119439369DB0305D5436940242343BA
:105BC0004361A0020143916110BD0000002002402A
:105BD000E015002070B5054600F018FC0646184C8C
:105BE0000AE0681C08D0002D04D000F00FFC801BD8
:105BF000A84201D9032070BDA069C007F1D1A069F6
:105C0000800701D50220A061A069C00511D4A06958
:105C100080050ED4A06940050BD4A069000508D406
:105C2000A069800405D4A069800302D4A069C003E0
:105C300003D5FFF787FF012070BD002070BD000075
:105C400000200240F8B51746002605460C4600F035
:105C5000D9FA09E029460220226800F0B5FA0028A6
:105C600004D1241D2D1D361DBE42F3D300F09EFA33
:105C7000BE4201D20020F8BD0120F8BD10B5084990
:105C800002460020054B497905E044001C5B944224
:105C900003D0401CC0B28842F7D310BD761200205A
:105CA0004000002010B5094800F020FD80B2FFF749
:105CB000E5FC074A074BFFF7DBFB0022064BFFF72B
:105CC0003FFCFFF721FD80B210BD00000C14002046
:105CD000F853E3A59B843E4000408F40F8B5414C0B
:105CE000E079002801D0002000E00120E0713D496A
:105CF0003D48CA790275097A41753C490A780276AD
:105D0000497841763A4801783748133001700521C7
:105D10004172962003F040FC4B20C00003F056FC7B
:105D20003149002213310C2003F020FD00210C200A
:105D300003F02EFD022003F07FFC2E4D00210F20EA
:105D400003F050FB2842E062F8D0E06A411C3BD0EF
:105D5000294E2A4F400439D58122D20100210F203B
:105D600003F0D9FC0021102003F03CFB41061E4843
:105D7000490E0022633003F06BFB1B4D6335687ADC
:105D8000052820D102221949681DFFF71BFA0028B7
:105D900019D1A87A607113480422691C4030FFF7BA
:105DA000EDF9206C00F02EF8A083607929464200BE
:105DB0000B3108467330FFF7E1F9A08B3188484377
:105DC000388002202070F8BD01F030FD0C480188B9
:105DD000A08B0546FFF78CF93088414339806D1E52
:105DE000A583F8BD4000002095110020E0000020B0
:105DF000B700002000D02724C2000020C0000020EF
:105E0000C400002010B504460E4800F06FFC0E4997
:105E1000C006C00E098805E02246C240D2070FD056
:105E2000401CC0B28842F7D3012005E02246C240A0
:105E3000D20705D0401CC0B28842F7D3491EC8B271
:105E400010BD00000C140020C4000020F8B5012093
:105E500003F015FB2A4CE084C0B2AD38FFF7E8FB35
:105E60002849FFF715FAFFF76DFC274A274BFFF784
:105E70004DFAFFF77BFC2649002760630546A063C7
:105E8000884238DB6078234E00280ED067702846A1
:105E9000FFF758FC00223346FFF7DCFA00221E4BC6
:105EA000FFF7E6FAFFF762FCA0622846FFF74AFC1C
:105EB00000223346FFF7CEFA184A194BFFF7D8FAFB
:105EC00005460E46A06AFFF73DFC144A154B5242A8
:105ED000FFF7CEFA2A463346FFF718FAFFF746FCDB
:105EE0001149A062884201DDA16204E0FF21C905D9
:105EF000C84200D3A762A06AFFF7CEFBC0B2F8BDCC
:105F0000B400002000002D436666666666660A409F
:105F1000000040400000084000E064403333333369
:105F200033B33040CCCCEC3F0000C84270B5002405
:105F3000014620314A79022A03D00421C163012499
:105F400018E0026813680E25AB43136002681368FB
:105F50005B085B001360436C1C2213400122154652
:105F60009D40036C5D604A7100220A71816B0029BB
:105F700000D08847204670BDF0B4016C0D68016800
:105F80000C68466C1C2304221E401746B7402F4263
:105F90000ED067070CD50C68A40602D40C68944395
:105FA0000C60416C19408A40016C4A60016B1AE038
:105FB0000227B74002462F402032002F17D0A707F4
:105FC00015D50C68A40605D40C680A25AC430C60F2
:105FD00001215171446C02211C40036CA1405960A5
:105FE00000211171C16A002918D0F0BC08470827A8
:105FF000B7402F4212D0240710D50C680E25AC43B1
:106000000C60446C01211C400B46A340046C63608F
:10601000C163517100211171416BE4E7F0BC70471D
:1060200070B504003CD01F48256814212818FFF7DC
:106030005FF8800060641C48206402212046203004
:106040000246417129681948E3680140A068666901
:106050001843236933431843A3691843E36918437A
:10606000236A1843084328600121A06889038842F5
:1060700010D00D488030836A656C1C210D400F26BE
:10608000AE40B3438362656C63680D40816AAB4088
:106090000B4383620020E06301215171107170BDD8
:1060A000012070BDF8FFFDBF000002400F80FFFF20
:1060B000F8B504468C46203001790025012909D025
:1060C0000126067141790027012905D007710225B3
:1060D0002846F8BD0220F8BD02214171E76320681F
:1060E000016849084900016061462046FFF76EFCDF
:1060F000206B00282068016801D00E2205E00422F0
:1061000091430160206801680A2211430160206800
:10611000016831430160DBE770B5044600F076F9B1
:106120000546601C00D0641C00F070F9401BA042C2
:10613000FAD370BDF8B51A4E0546307C0F460128DB
:1061400007D0012030741748FFF744FD010002D04A
:1061500021E00220F8BD0020C04338606C6814E0E4
:106160002046FFF7B5FC0F48FFF734FD01460E4807
:10617000426808239A434260426843159A4342604A
:10618000002901D03C6006E08034A8686A68C0013C
:106190008018A042E4D8002030740846F8BD000002
:1061A000E015002050C3000000200240054841686F
:1061B00002221143416041680122114341600020E5
:1061C0007047000000200240F8B50C4C1646207CB9
:1061D0000F46012808D0012020740948FFF7FAFC77
:1061E0000025002802D006E00220F8BD65613E606F
:1061F0000348FFF7EFFC2574F8BD0000E015002010
:1062000050C3000011484168C9070BD0EFF310815B
:1062100072B60F4AC2600F4AC26081F310884168AB
:10622000C9070ED1416889070DD5EFF3108172B609
:10623000094A0261094A026181F3108840688007B7
:1062400001D5012070470020704700000020024067
:10625000EFCDAB8905040302BFAE9D8C1615141358
:106260007047000010B504494A69024202D04861F3
:10627000FFF7F6FF10BD000000040140F8B5002351
:106280000124A2E027469F403A4070D04D68022D7D
:1062900001D0122D14D1DD08AD002D1800952D6A06
:1062A0005E07AC46F50E0F26AE46AE406546B543DA
:1062B000AC460E697546AE4065462E43009D2E6283
:1062C0004D68012D05D0022D03D0112D01D0122DC6
:1062D00016D185680326AC465D00AE46AE406546E5
:1062E000B543AC46CE687546AE4065462E438660E3
:1062F00046680D79BE43ED06ED0F9D403543456080
:1063000006685F000325BD40AE46AE430D79B44636
:10631000AE07B60FBE4065462E430660C66875469A
:10632000AE438D68BD403543C5604D68ED004BD52B
:10633000294D6E6B26436E639E08284DB600751975
:10634000AC46AD689E07360F0F27B740BD43052703
:106350003F07B84201D1002715E0214FB84201D1D3
:10636000012710E01F4FB84202D102270BE02BE0BB
:106370001D4FB84201D1032705E01C4FB84201D19F
:10638000052700E00627B7402F436546AF60184D4C
:106390002E684F689643FF0300D516432E606E6843
:1063A0004F689643BF0300D516436E60AE684F68D2
:1063B0009643FF0200D51643AE60EE684F689643E1
:1063C000BF0200D51643EE605B1C0A681546DD402F
:1063D00000D057E7F8BD0000001002400000014067
:1063E0000004005000080050000C0050001C005039
:1063F000000401400069084000D001207047002AD5
:1064000001D08161704781627047000001480068D7
:1064100070470000FC00002002480168491C016030
:1064200070470000FC00002010B5084800240168F7
:10643000402211430160204600F00AF8002801D0F4
:10644000012401E000F07EF9204610BD002002404A
:1064500070B5054609487D210024C9000068FEF793
:1064600047FE00F0E9FD002801D0012404E00022ED
:106470002946501E00F07CF9204670BD0001002026
:1064800070477047F8B5294CA078401CA0700120D7
:106490002071608C401C6084A08901F089FE244D2D
:1064A000E888FFF7D0F8234F3946FEF7F1FE224E79
:1064B00000903168FEF793FE30600120216BC0052B
:1064C000814203DB0098FEF7DFFE20631B4E0221B2
:1064D0003046FFF78FFF002802D00020E063F8BDB0
:1064E000E888FFF7B0F83946FEF7D2FEE16BFEF719
:1064F00076FE1349E0638842F1DB207A002813D04E
:1065000000210B484030818003F06AFA012100220B
:1065100089023046FFF773FF7D200001FFF7FCFD85
:1065200009490848C860F8BD0121EAE7B400002025
:10653000340D002000007A44F800002000040050D0
:106540000000A0400400FA0500ED00E0704770472D
:10655000704710B5044600680168C943C90708D1EF
:106560008168C943C90704D1012141602046FFF772
:1065700089FF20680168C943890708D48168C94335
:10658000890704D4022141602046FFF779FF206883
:106590000168C943490708D48168C943490704D43D
:1065A00004214160204600F0CBF820680168C9430F
:1065B000090708D48168C943090704D40821416048
:1065C0002046FFF7C3FF20680168C943C90608D405
:1065D0008168C943C90604D4102141602046FFF7F1
:1065E00050FF20680168C943890608D48168C943FF
:1065F000890604D4202141602046FFF7A9FF2068C6
:106600000168C943490608D48168C943490604D4CE
:10661000402141602046FFF79AFF10BDF8B5040005
:1066200005D025462035A87B002802D006E00120B1
:10663000F8BD00206873204600F040F80220A873DF
:106640002068C26884466368012B04D00120A16AD7
:10665000C005814201D11E208243154861698142F3
:1066600001D0144802401448A6680240184630433E
:10667000676A266A3E433043A66A30431043012BC3
:1066800003D00122D205964203D12369E2681A435E
:106690001043074A914205D0A2691143E2690243BF
:1066A000084610436146C8600120A8730020F8BD69
:1066B000FFFF00003F1FFFFFF8F119FF10B5006852
:1066C000084988420CD10848816BC2041143816398
:1066D000002201210D2000F04BF80D2000F03EF8C3
:1066E00010BD0000007C0040001002400068C0693E
:1066F0007047000070B50224034620339C730F4C92
:106700002568E604354325600468E568B61235431C
:10671000E5600568AE6801242643AE6005682E6911
:1067200026432E610568A96101684A610068016914
:106730000422114301619C73002070BD00040140DC
:10674000704700000448416B012211434163816B93
:10675000020411438163704700100240C106C90E54
:1067600001208840014908607047000000E100E016
:1067700010B501F039F810BD0248016882151143C7
:1067800001607047007000400A4B1A68920892003E
:1067900002431A6008480369042213430361012974
:1067A00006D040BF20BF20BF0169914301617047FF
:1067B00030BFF9E70070004000ED00E0F8B5044696
:1067C0000078544D800672D5524E0027403EB06B83
:1067D000C00004D4B06BA9050843B06301274E483C
:1067E0000168C90511D40168821511430160FFF7E2
:1067F0000DFE009005E0FFF709FE0099401A64289D
:1068000037D845480068C005F5D532680321090529
:1068100060680A400140914208D08103890F032932
:1068200004D13168890301D50120F8BD2A6903210B
:1068300009040A4022D0084090421FD020788006E8
:106840001CD528692A6988430121C9040A432A61A1
:106850002A698A432A612861C0050FD5FFF7D6FD52
:10686000009008E0FFF7D2FD0099411A2B488142C1
:1068700001D90320F8BD28698005F3D56168880334
:10688000800F032805D132680005824301400A4386
:1068900032602869032261681204114008432861AC
:1068A000002F04D0B16B012000078143B163207831
:1068B000C00705D0E868A168800880000843E86048
:1068C0002078800705D5E8680C218843E1680843F3
:1068D000E8602078400706D5E868032189028843EC
:1068E00021690843E8602078000706D5E86803219D
:1068F0000903884361690843E8602078000606D5EB
:10690000E868032189048843A1690843E8600020FE
:10691000F8BD0000401002400070004088130000E5
:10692000F8B50E4605007DD053480068C007C00F7B
:10693000B0420AD250480168490849003143016019
:106940000068C007C00FB04271D128784B4C800757
:1069500005D5E068F0218843A9680843E0602878FD
:10696000C00752D06868022817D0032818D02168C1
:10697000012818D08905002959DAE16889088900B9
:106980000143E160FFF742FD69680746022912D022
:1069900003291CD0012926D033E021688903EAE7C6
:1069A00021688901E7E74907E5E7FFF72FFDC11BEC
:1069B0003348814223D8E0680007800F0228F4D1D1
:1069C00023E0FFF723FDC11B2D48814217D8E06863
:1069D0000007800F0328F4D117E0FFF717FDC11B54
:1069E000274881420BD8E0680007800F0128F4D1C6
:1069F0000BE0FFF70BFDC11B2148814201D90320A9
:106A0000F8BDE0680007800FF3D11B480168C90793
:106A1000C90FB1420DD901684908490031430160ED
:106A2000006800E003E0C007C00FB04201D00120C1
:106A3000F8BD2878400706D5E06807210902884399
:106A4000E9680843E0602878000707D5E068072177
:106A5000C90288432969C9000843E06000F036F89C
:106A6000E168084A0906090F515CC84006490860F8
:106A70000020FFF7EDFCF8BD0020024000100240AE
:106A800088130000DE9A0008000100200448054930
:106A90000068C968044A4905490F515CC8407047FD
:106AA0000001002000100240F79A00080448054940
:106AB0000068C968044A8904490F515CC84070479E
:106AC0000001002000100240F79A000810B5184A93
:106AD000D1680C20084004280BD0082810D00C28BE
:106AE00010D050680004410F0120C003491C8840A9
:106AF00010BD1068C00601D50E4810BD0E4810BD6F
:106B00000E4810BD88020E4B000F185C0902D368B6
:106B1000890F491CDB0301D5084A05E01268D2063B
:106B200001D5044A00E0044A5043FEF7E1FA10BDE3
:106B30000010024000093D000024F40000127A0019
:106B4000EE9A0008FEB505007ED0FE4CE7680C20EA
:106B5000E66807400120000406402878C00747D0B7
:106B6000082F05D00C2F0AD101200004864206D13F
:106B7000206880033CD568680028E5D038E0012013
:106B800069680004814203D121680143216011E05A
:106B9000052301221B0492049942216802D111436A
:106BA0002160F1E781432160216801400091206864
:106BB00090432060686800280DD0FFF727FC009004
:106BC00005E0FFF723FC0099401A64287AD8206872
:106BD0008003F6D50CE0FFF719FC009005E0FFF705
:106BE00015FC0099401A6428F0D820688003F6D478
:106BF0002878800755D50923E868042F0DD00C2F7D
:106C000001D1002E09D000283BD0216899430143CF
:106C10002160FFF7FBFB064627E02168490701D505
:106C2000002891D061681F22120291432A69120242
:106C3000114361602168994301432160FFF746FFDA
:106C4000E16809060A0F00E079E1BF49895CC840A4
:106C5000BE4908600020FFF7FBFB002872D120E04E
:106C6000FFF7D4FB801B0228B0D820684007F7D577
:106C700060681F210902884329690902084360608E
:106C80000FE02068400840002060FFF7BFFB064689
:106C900004E0FFF7BBFB801B022897D82068400761
:106CA000F7D42878C0065FD5002F0CD0A86900283B
:106CB00049D02068FF21013108432060FFF7A6FB7F
:106CC00006462DE0C0E02068800502D5A8690028AE
:106CD000A7D06068072149038843296A0843606098
:106CE0006068297F0002000A090608436060286A7C
:106CF000410B0120C003491C8840E16809060A0FC6
:106D00009149895CC840914908600020FFF7A0FBC9
:106D1000002817D128E0FFF779FB801B0228A3D8B1
:106D200020688005F7D56068072149038843296AF0
:106D3000084360606068297F0002000A0906084372
:106D4000606011E0E1E02168FF20013081432160B3
:106D5000FFF75CFB064604E0FFF758FB801B0228A8
:106D600072D820688005F7D42878794E000724D59A
:106D700068690028306910D0012108433061FFF7AD
:106D800045FB009005E0FFF741FB0099401A0228FF
:106D90005AD830698007F6D50FE0400840003061CE
:106DA000FFF734FB009005E0FFF730FB0099401A35
:106DB000022849D830698007F6D42878400765D57D
:106DC00000200290A06BC00006D4A06B012109072F
:106DD0000843A063012002905E480168C90511D4F0
:106DE0000168821511430160FFF710FB009005E078
:106DF000FFF70CFB0099401A642825D85548006815
:106E0000C005F5D5FF20AA680130824203D131695F
:106E10000143316111E001218902002A07D00523D5
:106E20001B029A4203D132690A433261EFE73269A9
:106E300082433261306988433061A86800280FD0EE
:106E4000FFF7E4FA009007E05EE0FFF7DFFA009951
:106E5000411A4148814257D830698005F5D50DE087
:106E6000FFF7D4FA009006E0FFF7D0FA0099411A34
:106E70003948814248D830698005F5D40298002805
:106E800004D0A06B012109078843A063686A002829
:106E900064D00C2F3ED0012636060228206805D08B
:106EA000B0432060FFF7B2FA05462FE0B043206000
:106EB000FFF7ACFA074604E0FFF7A8FAC01B022868
:106EC00022D820688001F7D4E96AA86AE2680843FA
:106ED000296BFD231B049A4311430843E06020689B
:106EE00030432060FFF792FA054604E0FFF78EFA80
:106EF000401B022808D820688001F7D52EE0FFF754
:106F000085FA401B022801D90320FEBD20688001BC
:106F1000F5D423E00128F8D0E06801210904AA6A29
:106F2000014091420BD10F218904EA6A014091424C
:106F300005D1032189050840296B88420ED0012024
:106F4000FEBD000000100240DE9A00080001002093
:106F50004010024000700040881300000020EFE75E
:106F600070B5040007D0002625464035A662687C2F
:106F7000002802D005E0012070BD2E74204600F0EC
:106F80002FF8022068742068016840229143016054
:106F9000A168606822690843E16811430843616998
:106FA00001220843A169520211400843E1690843E4
:106FB000216A0843A16A084321680860A069042186
:106FC000000C0840616A0843216848602068C16974
:106FD00092009143C161666501206874002070BD14
:106FE00010B586B0044614216846FEF7E0F8104953
:106FF0002068884219D10F48416B821411434163C4
:10700000C16A01221143C162C06A0021104005908B
:10701000E02000900220019003200390029104914F
:10702000052069460007FFF729F906B010BD0000EA
:107030000030014000100240094910B5401E88424E
:1070400001D9012010BD074C60610321081F00F029
:10705000CBFB0020A06107202061002010BD0000B4
:10706000FFFFFF0000E000E070477047F8B50268DE
:107070000446D0691168936805072D0F5BD0DD07C2
:10708000ED0FFF2621360E402E4367D0C60706D0EF
:10709000CE0504D501261662E26F3243E267870708
:1070A00002220426002F06DADF0704D027683A629E
:1070B000E76F3743E767470706D5DB0704D0236848
:1070C0001E62E36F1343E367020709D520220A40DB
:1070D0002A4305D0236808221A62E36F1343E3674B
:1070E000E26F002A2FD0800606D5880604D5216ECF
:1070F000002901D020468847E06F21688968490649
:1071000001D4000724D5204601F09AFA206881684E
:10711000490619D58168402291438160E06E0028BC
:1071200012D020498163E06EFEF700FF00280AD0EC
:10713000E06E816B06E0850610D58D060ED5216EBA
:107140001CE020468847F8BD2046FFF78EFFF8BDBB
:107150002046FFF78AFF0020E067F8BDC50208D58A
:107160005B0206D50120000510622046FFF77CFF78
:10717000F8BD030605D50B0603D5616E0029E0D1E5
:10718000F8BD4006FCD54806FAD5136820464021D4
:107190008B431360202161670021616600F069F96B
:1071A000F8BD00009D85000810B5040003D0606F95
:1071B000002802D007E0012010BD002170200155F9
:1071C000204600F027F824206067206801684908FD
:1071D00049000160204601F07DFA0128ECD0606A88
:1071E000002802D0204601F0BBF82068416809223F
:1071F000D20291434160206881682A2291438160D4
:1072000020680168012211430160204601F00EF957
:1072100010BD0000F0B587B0064614216846FDF7A2
:10722000C6FF2C493068884251D12B48416B01225E
:10723000920311434163C16A01221143C162C06AD2
:1072400000251040059003204002009002200327F3
:1072500001A9A1C104200490052069460007FFF799
:107260000DF81F4C1D48A560E56081C48027E560CE
:10727000A7602020256160610002A0611848083CD9
:10728000FEF7CEFE002801D0FEF720FCF466A662D1
:10729000144C1248214614382060032060601020EE
:1072A0000831A1C16561A561E56120462562FEF74F
:1072B000B7FE002801D0FEF709FCB46600220121C8
:1072C0001B20A662FFF754FA1B20FFF747FA07B00E
:1072D000F0BD0000003801400010024030000240C4
:1072E0005015002098150020F8B50446806F20281E
:1072F0004DD100290BD0002A09D00123A0681B031F
:10730000984206D12069002803D1C80701D0012086
:10731000F8BD25466035287C012838D00120287426
:107320005820616502530026E6672220A067E06EC0
:10733000002819D01749C162E16E17480863E16E51
:1073400016484863E06E13468663676D21683A46C7
:107350002431E06EFEF7ACFE002805D01020E06777
:107360002E7420206067D2E72E7420680168FF2207
:10737000013211430160206881680122114381605C
:10738000206881684022114381600020F8BD0220FE
:10739000F8BD0000F985000837860008B1850008AF
:1073A00070477047FFB50446406F83B017460D46DF
:1073B00020285CD1002D0AD0002F08D0A168C00180
:1073C000814207D12069002804D1E80702D00120BA
:1073D00007B0F0BD204660300290007C012846D006
:1073E0000298012101740020E06721206067FFF707
:1073F0000DF8264640360190378277820120A16839
:107400000003814202D12069002802D02F460025C6
:1074100011E000270FE000228021204601F06EFAE3
:10742000002815D1002F15D02168387888627F1C7C
:10743000708A401E7082708A019B00280698009016
:10744000E9D100224021204601F058FA002808D056
:107450000320BDE728882168C005C00D8862AD1CE7
:10746000E6E720206067029900200874B0E7022058
:10747000AEE7704701490248C160FDE70400FA0524
:1074800000ED00E0F8B501F001F801F03BF83B48F1
:107490000068C0693A4E3B4F800700D5FE60FEF79A
:1074A00001FC0121C9023848FEF7A4FF374C002532
:1074B000002823D036480560E079002803D1012058
:1074C000E07101F079FA2078632806D900220821BA
:1074D0002D48FEF794FF012205E0012208212A48E9
:1074E000FEF78DFF002201210520C9030007FEF7EA
:1074F00086FF284CA08C012803D01CE0E5710022F7
:10750000ECE725486946088072B680212348FEF7DB
:10751000F5FA002804D0022269462048FEF792FBC3
:1075200062B61FA001F0E4FAA58402F059FA6420C3
:1075300001F0F4FCFE60608C012809D115486584D7
:107540004038058002F04CFA642001F0E7FCFE6050
:10755000208C012806D1258402F042FA642001F033
:10756000DDFCFE600B48124A40380188914202D18E
:10757000C088002800D1FE60F8BD0000D0140020B3
:107580000400FA0500ED00E000040050B400002003
:10759000F8000020740D0020AAAA0000384A000854
:1075A000BDF8C8EBC9FDBCB6C4A3CABD0D0A000036
:1075B000AA55000010B50248FEF7CBFF10BD000031
:1075C0000C14002008B50848016B01221143016327
:1075D000006B01211040009000220A20FFF7C8F83C
:1075E0000A20FFF7BBF808BD00100240F0B587B0D5
:1075F00014216846FDF7DBFD4748C26A04210A43AF
:10760000C262C26A0A400592C16A80263143C162E1
:10761000C16A31400591C16A01242143C162C16A36
:1076200021400591C16A02252943C162C06A2246F0
:107630002840059005201C210007FEF7E0FE0122EE
:1076400036493748FEF7DBFE002236493448FEF75C
:10765000D6FE91210520002209020007FEF7CFFE89
:1076600031480190002705206946029700940007E1
:10767000FEF704FE0C2000901120019003200390DF
:107680000520029769460007FEF7F8FD10206A46BC
:10769000039591C2052069460007FEF7EFFD112012
:1076A000019002976946039700941D48FEF7E6FD96
:1076B0001E4801906946009502941948FEF7DEFDC8
:1076C000E00200906946019702951548FEF7D6FD45
:1076D0001748694691C1694611480397FEF7CEFDE8
:1076E00091200002694691C1052069460007039771
:1076F000FEF7C4FD69460A48019700960294FEF71A
:10770000BDFD002201210520FFF732F80520FFF71B
:1077100025F807B0F0BD0000001002400102000093
:10772000000400500830000000001110000021107B
:107730000832000010B50F4C0D482060FF200530C6
:1077400060600020A060E06020616061E061012174
:10775000206249026062A161A0620720E0622046C7
:10776000FFF7FEFB2068016840221143016010BD55
:10777000003001403C14002000B585B0142168465B
:10778000FDF715FD164815490160E12149024160E8
:1077900000218160C160016181610C22C16142618F
:1077A0000162302141620121090381634900C16303
:1077B000FFF7FAFC012080020090022001900120D6
:1077C00002900320039004200490052069460007DE
:1077D000FEF754FD01F0EAF805B000BD00380140A5
:1077E000D0140020704700008307FF22DB0E9A4070
:1077F0008907090E994000280BDA0007000F0838A6
:10780000830808489B001818C36993430B43C3615E
:107810007047830804489B001B181868904308436E
:107820001860704700ED00E000E400E0BFF34F8F08
:1078300004490348C860BFF34F8F00BFFDE7000055
:107840000400FA0500ED00E0F0B58DB0962001F0DF
:10785000A3FEFE4801F0BAFEFD4F00247C70B87B09
:107860000C2801D30B20B873012205205102000718
:10787000FEF7C5FDB87B78737871F648BC70F64D9D
:1078800000782870F548022100782871F448FEF746
:10789000B1FD00285FD00020B979EF4D49000843C1
:1078A000E871B86AE870401CB86278792946A87215
:1078B0004200CE310846C338FDF760FC06202A4658
:1078C0006872133AE2490492887F1075C87F507538
:1078D00078790022400029460D3001F047FF787981
:1078E000002140000D3001F053FF022001F0A4FE02
:1078F000EC713C74BC7201203873FC72D948FEF7FD
:10790000F5FE78840546BC707879FDF7B7FED64A57
:10791000D64BFDF7ADFD01F09DFA0022D44BFDF7EB
:10792000F5FCFDF7F1FE0006C10C481980B20121FB
:10793000C903B884884201D3401AB884CD4878631B
:10794000F878401CF870C748FEF7D0FE3884C2486B
:107950004E300990F6E101209EE7C248FEF7C6FED0
:107960003884C54DC54E21E0B87A002813D001F007
:1079700080FD069988420ED9059988420BD201F004
:107980004FFC3C73079801F000FE012001F054FE0B
:107990003872BC7211E0B348FEF7A8FE80B238849A
:1079A000B98C884202D38919884206D300210F205E
:1079B00001F018FD2842F862D6D0F86A411C1ED0AA
:1079C00040047DD58122D20100210F2001F0A3FEC9
:1079D0000021102001F006FD41069F48490E0022BB
:1079E000503001F035FD002001F0F0FD002001F0E5
:1079F000A2FD994D5035687A0728ABD101E0FFF719
:107A000015FF02229E49681DFDF7DCFB0028A1D16D
:107A10009148503001788F48007881429AD10026F1
:107A200035460AA801F07FFD04200AAA310E2D0276
:107A30000D433102165C0E43401EF7D5BE64FD6453
:107A400000263546104601F00CFD04200AA9320E2E
:107A50002D02154332020E5C1643401EF7D53E65DB
:107A60007D65B9786A46491CB9707B494D310D79FD
:107A700015704E7969464E70787B002809D1012235
:107A800075483A710988CE3001807A71049805757D
:107A9000467571486946CE30008809880091884251
:107AA0007ED109997748098A01806B4868494C3032
:107AB000808A48836B48FEF719FE3D46388400E013
:107AC00035E1788B7049FF30C33080B278838842CB
:107AD0000CD9494240186B49688308886A4A401C9F
:107AE00080B20B320880904200D30C80674903209B
:107AF00008700998564A81891186C089634B50865F
:107B0000903B2A6B1A601A46B03AD37C1E07360F98
:107B1000032E00D06E741A09AA74EC7001264C4A28
:107B2000AE729186D0866879FF21913148435649DB
:107B30002A6D593940180104C8176B6D89185841CE
:107B40000206080A1043524907904018069019216E
:107B500007988902401805900798B043010E00026B
:107B6000E965A8653C48EB6C0A30AA6C01F036FE6A
:107B700039486B6D16302A6D01F030FE3648EB6DDA
:107B80001230AA6D01F02AFE3348082141723149B2
:107B900000220978017068792F4980001C3000E0CC
:107BA00082E001F0E3FD6879002180001C3001F0E3
:107BB000EFFD29492648EE72042251314030FDF78D
:107BC000DDFA3048698B06887D20C000704340187C
:107BD000A8630A902F480078E87300902E48C08868
:107BE000FDF731FD02903046FDF72DFD0299FDF7BE
:107BF0004FFB7F21C905FDF7F2FAFDF74DFD81B27C
:107C0000244801800098401E814201D10120E87281
:107C1000EE841420285EFDF71DFD00910890288C4D
:107C2000FDF72CFD1D4A1E4BFDF722FC029003912F
:107C30000A98FDF70FFD039B029AFDF70BFC009BD2
:107C4000089AFDF763FBFDF73BFD2BE010270000D2
:107C500040000020B7000020A8110020B400002040
:107C6000000400500C140020666666666666E63FF7
:107C700000000840A086010000D02724983A0000A8
:107C8000E0000020F4000020E7030000381300208B
:107C900000AEFCFFD6000020340D0020F853E3A511
:107CA0009B843E40E8634DE00846FDF7E7FF797BA3
:107CB00088420BD301223A717A79521C7A719D4A1B
:107CC00043000099D15204990D754E75994A0321CC
:107CD000C23211540999984A8B891386C9895186F1
:107CE000810094483A6B32304250B038C07C7B7C83
:107CF0000207120F3D469A4202D9032A00D0687447
:107D00008C486B6DCE38081816302A6D01F066FD70
:107D10006879884980000022CE391C3001F026FDA8
:107D20006879002180001C3001F032FD0AE02A460B
:107D300000210F2001F0EFFC387B002802D000204A
:107D400001F0F9FB398CB88C814200D205E67B4A00
:107D500080188142FAD87A48008881004018F97862
:107D6000884200D27C74774A00210F2001F0D3FCB6
:107D7000B8787871F878002501280BD97248FEF799
:107D8000B5FC7249C9880901FDF7B2F9704802884B
:107D9000891801800020B8737A7B3979521821E064
:107DA000644BC233195C00291AD0BC7BAB00641C45
:107DB000BC73604C9C469234E1505E4B44006E00B4
:107DC0001C5B18339C5384001A335A4E1C5963466B
:107DD0006236F4506D1C33466033491EEDB21954BF
:107DE000401CC0B28242DBD8B878032801D2B87BED
:107DF000B87351490022887B48730490401E32E0DA
:107E000000212CE04B4C8B0062341E19B446E5581F
:107E10007668B54221DD0695464D4C0018352D5B40
:107E20009700AE46434D9235ED590595414D62356B
:107E3000EE504A3D3F4E67197D881836355334461B
:107E40007A341E193B4D74689235EC506346069D9A
:107E50005D6075467D80059D7560491CC9B2814293
:107E6000D0DB521CD2B28242CADB334C002060729B
:107E7000049B2AE02F4A41001832555A183A5552AD
:107E80008C4615468100623516466D58323675505F
:107E9000304EB54217D0154692356D58032D12D18C
:107EA000677A06263D46754316461A3E6244AD196A
:107EB0001288AA8032464C3289180A88EA8049889A
:107EC00029817F1C6772401CC0B29842D2D3194DE1
:107ED00055201A3D2870AA2068700420A870617A85
:107EE00006204843811CE970A81CFDF755FD20833E
:107EF000617A062251434A1990802846891D00F074
:107F000049FD00202946134A4C318300401CC0B271
:107F1000CA500C28F9D30B4A002180320F2001F0FF
:107F2000FAFB01210520002249020007FEF767FA4B
:107F30000DB0F0BD7612002040000020983A0000FD
:107F4000C800002000D027240C140020340D00208D
:107F5000BE000020FFFF010070470000FEB544494D
:107F60004248086001F0DCFC424800F0E1F8424C75
:107F700060834048801C00F0DBF8A0833D48001D72
:107F800000F0D6F8E083FF203C4D2630688028467C
:107F90004030017921720291E88E3949C0B20870EF
:107FA0000190E88F6071A88FA071A87AE070A8880E
:107FB0000090E0622889FDF761FB324A324BFDF701
:107FC00057FA00F047FF0022304BFDF79FF9FDF70D
:107FD0009BFB86B2E681EF8831463846FDF788F88C
:107FE000208201460098FDF783F871438EB27D2010
:107FF000C000A6817043FDF741FB254A254BFDF7E4
:108000009FFAFDF781FB60827D20E6823946C00041
:10801000FDF76EF8A0822084688F607202990120BB
:10802000002902D160710A216172002F01D16421FF
:10803000E980019A1249432A01D943220A706084D7
:10804000FDF730FE2083628A13491448FEF752FB85
:1080500013A0E16A00F04CFDE98815A000F048FD8E
:10806000298918A000F044FDFEBD0000E589000844
:1080700038000020004F0008B4000020340D00201C
:1080800000000020666666666666E63F00000840FF
:10809000F853E3A59B843E40FF7F00000C140020B2
:1080A000B1EAC7A949443A202564202E0D0A0000F0
:1080B000CDA8D1B6BCE4B8F43A202564206D732E67
:1080C0000D0A0000B5A5B4CECDA8D1B6BBF9D5BE7A
:1080D000CAFDC1BF3A202564B8F62E0D0A00000083
:1080E00070B586B014216846FDF761F801250F4E82
:1080F000ED03002229463046FEF781F901200024D5
:10810000019002946946009503943046FEF7B6F854
:108110000320019002946946009503943046FEF7CF
:10812000ADF8022000F0FAFE06B070BD0004005069
:108130000088704770470000F8B5044600206A4682
:108140001080194D55222A70AA226A700322AA7043
:10815000661DEE702A716971144A49008918AC7164
:108160002246E81DFDF70AF8002007E029186A46B4
:108170008978128889186A461180401CB042F5DB64
:10818000611DA81CFDF708FC0146684601802919FD
:108190000078C87168464078087221460931024863
:1081A00000F066FAF8BD0000A8130020340D00208E
:1081B00070B50F48C088FDF761FA0E4A0E4BFDF707
:1081C00057F90E4E04460D467089FDF757FA2246C0
:1081D0002B46FDF79BF8FDF773FA094A510C00E0B6
:1081E00080188842FCDC074970810968486170BDCD
:1081F000340D0020FCA9F1D24D624040B4000020B3
:108200000180FFFF0C140020034A1168382389B253
:1082100099430143116070470030014010B5FEF7EB
:10822000FBF810BD10B59AB034216846FCF7BFFFCB
:1082300014210DA8FCF7BBFF1C2112A8FCF7B7FF07
:108240001B4801680324E402A143C2148918016099
:10825000FEF792FA17480169A143016106200090D8
:10826000FF20013002900120039010200490022092
:10827000099040040B90000100240C900A94684679
:10828000FEF760FC0F200D9003200E900F941094C9
:10829000012111940DA8FEF743FB812012900320C9
:1082A00080041890149412A8FEF788FA1AB010BD32
:1082B00000700040401002401048016882151143D0
:1082C0000160C1680E4A1140C16001680D4A114049
:1082D00001608168490849008160016801229204B7
:1082E00091430160C168FD2212049143C1600021E5
:1082F0000161064904488860704700000010024090
:108300000C40FF88F6FFF6FE0050000800ED00E08C
:1083100070B501F07BF80F4C0F4D606402E001F086
:1083200075F86064A842FAD10020E0822078002825
:1083300009D0012802D0022805D102E0FDF7CEFCC9
:1083400001E0FFF781FAFDF781FD0449087000F0B4
:108350004FFF70BD400000203001CADEB400002095
:1083600010B5818CC90707D001684A6801235B04F6
:108370009A43836A1A434A60818C890707D501684A
:108380004A6801231B049A43C36A1A434A60818CDA
:10839000490707D501684A6801239B049A43036B88
:1083A0001A434A60818C090707D501684A6801238E
:1083B000DB039A43436B1A434A60818CC90607D595
:1083C0000268916801231B039943836B19439160F1
:1083D000818C890607D501688A6801235B039A436B
:1083E000C36B1A438A60818C490612D503685A68A8
:1083F00001210905046C8A4322435A60026C8A42B7
:1084000007D10268516803235B059943436C194304
:108410005160818C090607D501684A680123DB0495
:10842000806C9A4302434A6010BD0000F8B50026F4
:108430000446C667FDF7EAFF054620680068124F4C
:10844000000709D501212B46002249052046009747
:1084500000F054FA00280DD12068006840070BD5C1
:1084600001212B46002289052046009700F046FA9C
:10847000002801D00320F8BD20206067A067603489
:1084800026740020F8BD0000FFFFFF01F8B5184C6E
:10849000C826E078002829D16079002826D101205B
:1084A0006071144D686B002700281ED0686BC821CE
:1084B000081A15E01048E168405C616988470F4878
:1084C0000A21008848430E490880E068401CE060AB
:1084D000E068C82800DBE760696BC820401A761E98
:1084E000E168814201D0002EE4DC6771F8BD000034
:1084F00024000020000002406C0C0020C800002076
:10850000D800002070B5224CE07800283FD12079B7
:1085100000283CD1012020711E4EF169002509067A
:10852000002933DA2156625791420AD1F069400698
:108530002CD5A079002829D0A5712089401C208144
:1085400024E0A179002903D1A0710A2000F0EDFCFC
:1085500000202056CC2148430F49421820691218A8
:108560001279B262401C00222061A256CC235A43E9
:10857000895881420ADC25612078401C20702078CF
:108580000E2800D12570A078401CA070257170BD08
:1085900024000020003801404401002010B5806A0A
:1085A0000022014640314A834A82FEF75EFD10BD3B
:1085B00070B5846A606FA56F216889680026090616
:1085C000002906DA212804D152200653204600F063
:1085D00047F820688068400606D5222D04D15A202D
:1085E0000653204600F02CF8E06F10210843E067A6
:1085F0002046FEF73AFD70BD10B501460968806A55
:108600000968890614D400225A210A5201680A68AE
:10861000FF2301339A430A6001688A6852085200B6
:108620008A6001688A6840239A438A6020218167B2
:10863000FEF7B6FE10BD10B5806AFEF7B2FE10BDA3
:1086400001680A68FF2321339A430A6001688A6837
:10865000520852008A60202181670021016670471C
:1086600001680A68C0239A430A6020214167704765
:1086700070B5164CE278002A0CD12279002A09D173
:108680000122E2700025C82903DC0222A256002A3A
:1086900001DCE57070BD0123E356CC2253430C4A44
:1086A000D1500123E356CC2673439B180A4601465A
:1086B000181DFCF763FD6078401C607060780E2820
:1086C00000D16570A078401EA070E2E72400002071
:1086D00044010020F8B504462669A268E7693243E0
:1086E0006669102000253E432368324378491E689E
:1086F000784F3E4016431E6023685A6803263603AF
:10870000B243E66832435A602368A2698B4201D0C3
:10871000266A32439E680B273F02BE4316439E6083
:108720006D4E23686D4AB3420CD1D2689207920F06
:1087300006D0012A38D0022A34D0032A20D11EE0E4
:1087400001201DE0664EB3420AD1D2680C263240A9
:1087500026D0042A28D0082A24D00C2A10D10EE0D2
:108760008B420DD1D66803229202164018D0012206
:108770009202B61A18D0B61A14D0964200D1082028
:10878000564A0126403A574FF6038B4236D100280D
:108790000CD002280DD0042812D008281FD11CE0CC
:1087A0000020EDE70220EBE70420E9E7FEF76EF991
:1087B00008E01068C00601D5384605E04A4803E0E5
:1087C000FEF784F9002873D0626851005118814285
:1087D00005D81103814202D303E03046F4E70125B6
:1087E00066E0010E06025008002330185941FCF7DC
:1087F00095FC03210902411A3C4A55E0E169B14266
:1088000032D1030000F09BF909070A0D0625060680
:10881000062B0600E3E7FEF739F91CE0FEF746F900
:1088200019E010686168C00602D54808304A01E0C6
:10883000304A48088018FCF75BFC80B201462E4A9B
:1088400010399142CBD8511C01400007400F08431A
:108850002CE0FEF73BF9616840004A08EAE76168EE
:10886000012248081204E5E7030000F068F909074F
:108870000A0D06260606062C0600B0E7FEF706F9E6
:108880001DE0FEF713F91AE010686168C00602D512
:108890004808C01902E014484A081018FCF728FCE0
:1088A00080B20146144A1039914298D82168C860B4
:1088B0000020206660662846F8BDFEF707F961686B
:1088C0004A088018EAE7616848088019E6E700006E
:1088D00000480040F369FFEF0038014040100240BB
:1088E0000044004000093D000024F400FFFC0F009C
:1088F00000127A000048E801EFFF0000FFB581B0E8
:1089000017460E4604460A9D09E0681C07D0FDF78D
:108910007DFD0499401AA8420CD8002D0AD0206889
:10892000C1693046884318D00020B842EDD00020FD
:1089300005B0F0BD20680168FF22A13291430160BB
:108940002068816849084900816020206067A0672D
:108950000020603420740320EAE70120E5E70000EE
:1089600010B504491020096808620248FEF77EFB32
:1089700010BD0000D014002001B501231A4669463D
:108980000248FEF70FFD0248C06908BDD014002060
:108990000038014070B50D460646002403E0305D06
:1089A000FFF7EAFF641CAC42F9DB70BD01490D2002
:1089B000887070472400002010B507480A22818A79
:1089C00051438184FEF7FEFDFEF7D6FEC82203491F
:1089D0000348FEF789FC10BDB40000206C0C002099
:1089E000D0140020F8B53D4C002321783C4A1D46A8
:1089F000082910D0072945D006294ED0052950D086
:108A0000042951D0032952D0002954D0012956D02D
:108A1000022958D059E0A17800264A1F04E0304FBF
:108A2000BF5DFB189BB2761C9642F8DB667927790E
:108A30009A195118E3786278C9188918C919401829
:108A4000C0071AD0012E14D0022E16D12548244971
:108A5000C018FCF793FB00F0C3FF642000F05EFA3F
:108A6000BFF34F8F21492048C860BFF34F8F00BF2D
:108A7000FDE759081046FFF75FFB2570E570A5700C
:108A8000A571F8BDA1795054491CC8B2A071A17854
:108A9000491F8842F5D1082001E06070072020704E
:108AA000F8BDE0700620FAE760710520F7E7A070D6
:108AB000E5700420F3E7552807D10120EFE7AA2845
:108AC00003D10220EBE7032803D02570E570A570E1
:108AD000F8BD032020702071F8BD0000AB0000201D
:108AE00044130020340D00200400FA0500ED00E0DE
:108AF0000FB410B503A9044B044A029800F002F920
:108B000010BC08BC04B01847F59700080401002009
:108B10002021020C01D010211046020A01D010467B
:108B20000839020901D01046091F820801D01046F9
:108B3000891E420801D0881E7047081A704730B459
:108B40007446641E2578641CAB4200D21D46635DEA
:108B50005B00E31830BC184702E008C8121F08C1C8
:108B6000002AFAD170477047002001E001C1121FAE
:108B7000002AFBD1704708B50021684601706B469A
:108B8000012202212C2000F0D5FD0221684601704F
:108B90006B4601222C2000F0CDFD08BD38B50446FF
:108BA0006D20694608706B46012207492E2000F0AF
:108BB000C1FD0649002C01D0054A00E0054A2E20DF
:108BC00000F09EFD38BD00000608000006180000F9
:108BD000070600000716000038B504466B4602225F
:108BE0000021362000F018FCB3212300FFF7A7FF77
:108BF0000E0F08153A3A3A3A1C273A3A2F34483AB7
:108C000000216846017040784108490014E0694637
:108C1000087880088000401C04E0694608788008D5
:108C20008000801C08701DE0684602780A404832C7
:108C300002704178802001436846417012E0684626
:108C400002780A40027040784106490EF4E769460E
:108C500048780221084303E069464878FD2108402E
:108C6000694648706B4601220021362000F062FD03
:108C7000012200AB11463620013300F05BFD38BD08
:108C800069460878CF21084069462030CAE708B510
:108C9000032168464170012101706B4602220021C8
:108CA000362000F047FD0122D20306212D2000F0DE
:108CB00027FD012000F032F90120FFF78DFF08BDEC
:108CC00008B5020A69464A7008706B460222042100
:108CD0002D2000F02FFD0320694608706B4601220D
:108CE00006212D2000F026FD0020694608706B4605
:108CF000012206212D2000F01DFD0A212D2000F06B
:108D000071FB08BDFFB58DB00446002506E025289F
:108D10000AD0109A0F999047641C6D1C2078002887
:108D2000F5D1284611B0F0BD00270121484A00972F
:108D300000E00743641C23780846203B984010421B
:108D4000F7D120782E2817D1042007436078641CBF
:108D50002A280CD10E98641C02C800910E900BE0DA
:108D600000990A22514330394018641C0090207841
:108D7000014630390929F3D920780028D1D0642858
:108D800008D0692806D075281ED0109A0F999047F0
:108D90006D1C5BE00A200E99019001C90E9100281C
:108DA00002DA40422D2102E0390504D52B216A4622
:108DB0001172012103E0F90704D02021F7E70BAE7F
:108DC0000B910DE00021FAE70A200E99019001C9EC
:108DD0000E91F7E70199FCF78BF93031761E31706F
:108DE0000028F7D103A8801B20300190780701D517
:108DF000009801E0012000900199884201DD401AAD
:108E000000E000200027009006E002A8109AC05D54
:108E10000F9990476D1C7F1C0B988742F5DB04E08F
:108E2000109A30200F9990476D1C0099481E0090B1
:108E30000029F5DC05E03078109A761C0F999047F0
:108E40006D1C0199481E01900029F4DC641C65E743
:108E500009280100F8B54A002B4B520DD6182B4AB1
:108E60000C460546142E2BDA002E12DA284BFCF79E
:108E70004DFA00221346FCF769FD40D2002C03DABC
:108E80000124E40700253AE02046284337D0214C4E
:108E900014E0214F0B46F7403B402B4331D01C4B95
:108EA000FCF734FA00221346FCF750FD27D2002CC1
:108EB00003DD01200005F0400419BC4300251EE03D
:108EC000332E1EDC33460027143BFF43DF4038427D
:108ED00017D00F4BFCF7C4FA00221346FCF736FDFF
:108EE0000DD2002C0ADD142E0CD03420811B012061
:108EF00088404019A84200D2641C0546BD43214663
:108F00002846F8BD641CF9E701FCFFFF9C7500884A
:108F10003CE4377E0000F03FFFFF0F007D2110B5DD
:108F2000C900484300F001F810BD002140E000BF37
:108F300000BF00BF00BF00BF00BF00BF00BF00BF39
:108F400000BF00BF00BF00BF00BF00BF00BF00BF29
:108F500000BF00BF00BF00BF00BF00BF00BF00BF19
:108F600000BF00BF00BF00BF00BF00BF00BF00BF09
:108F700000BF00BF00BF00BF00BF00BF00BF00BFF9
:108F800000BF00BF00BF00BF00BF00BF00BF00BFE9
:108F900000BF00BF00BF00BF00BF00BF00BF00BFD9
:108FA00000BF00BF00BF00BF00BF00BF00BF491C23
:108FB0008142BCD370470000FEB5044600200190FA
:108FC00000906079734940000E5A61782578491EF7
:108FD0007148CFB20163042D77D0072D75D00021E1
:108FE0000291217801736C49E37901229205896924
:108FF000002B6CD0914381616748217A4173217ABB
:1090000082698907890B0A4382610021042000F0EC
:1090100082FB324661492E2000F072FB3846FFF792
:10902000BDFD5F4E0522705D810040185D4943180B
:1090300007212B2000F07EFB5B49029801220B18D0
:109040000B21282000F076FB705D584980000A58FB
:109050000C21282000F05FFBE07955498000401882
:10906000A1794900425A0221272000F049FB5148CA
:109070007E00825B0421272000F042FBE07900287B
:1090800029D0A07804282CD02820694608722022F4
:109090000621272000F034FB02AB012226212720E5
:1090A00000F048FB444938014018E17889004258F3
:1090B0000821272000F02FFBA17A601C627A0902A8
:1090C000114313D016E000E001E0012188E71143CD
:1090D000F608816190E764220621272000F010FB4A
:1090E000E0E71020694608720246D1E73349017271
:1090F000090A4172417A007A0A020243202127209C
:1091000000F0FEFA2E4F0C2123203A6800F003FBFA
:10911000F01982880421232000F0F2FAA0790028B7
:109120000BD0E0792749012243180021212000F0CB
:1091300001FB03200190012000902A07120F10016B
:109140000243607800218007000B0243019800056C
:1091500002430098400402432079C00640090243BC
:109160006079C00602431F2000F0D5FAA07861782C
:109170000123084302040848DB030261E179490343
:1091800019430A4302610021082000F0C4FA0020BC
:10919000FEBD0000AC9A0008080100200428000071
:1091A000549A0008010000201F0000205C9A00086B
:1091B0007C9A0008889A00088C9A000841100000E8
:1091C000749A00082100002038B50C4607498A8BA4
:1091D000002102432C2000F093FA684604706B468D
:1091E000012206212C2000F0A5FA38BD080100203C
:1091F00010B5FFF7C0FC10BD10B5044604213620A1
:1092000000F0F0F80121C902002C01D0084300E071
:10921000884302460421362000F07DFA10BD00008C
:1092200038B540206946087000210E2000F0DAF8B9
:109230000446002211460E2000F06DFA6B46012212
:1092400000210D2000F076FA074A00210F2000F0DF
:1092500062FA00F03BFA224600210E2000F05BFA91
:1092600002480021017338BDF8FF2724280100209F
:109270007CB505460420694608704B4C002060759B
:1092800021462031206348710873A0836063A06386
:1092900000F0BCF8454E206002E000F0B7F8206016
:1092A000B042FAD10020FFF797FC4148007824280B
:1092B00001D9243806E00621FBF71AFF0622101A0E
:1092C00040010843020601040A4301020A43024323
:1092D00000211E2000F01FFA6B46012200212420ED
:1092E00000F028FA1E20FFF7EBFC86B2300AA073CC
:1092F0000420FFF7E5FC0006000E0DD002206946B1
:10930000087101AB012212212D2000F013FAA08B6D
:10931000012109030843A08300F078F820600620AB
:10932000FFF7CEFC60600720FFF7CAFCA060F006E4
:10933000C00E207501D110202075C0B200F036FAA1
:10934000E80707D0FFF7A3FCA08B0121C90208435F
:10935000A0830AE00521362000F02EF815490840C8
:1093600002460521362000F0CBF90120FFF734FC3E
:109370000021042000F036F8A0610021262000F032
:1093800031F815218903084302460021262000F008
:10939000C2F900222621362000F0B2F900F036F89A
:1093A000206000207CBD0000080100203001CADEE2
:1093B00000000020FFFD000038B5094C89B280B2E2
:1093C0006B46022200F028F8002806D16846407853
:1093D000010268460078081884B2204638BD0000B3
:1093E000FFFF000038B50024E44389B280B26B4629
:1093F000042200F011F8002806D103216846435CDE
:109400002202D418491EFAD5204638BD10B50021D5
:109410000846FFF7E7FF10BD38B5002909D0402402
:1094200020436C462070C8B27F2906D860700220A5
:109430000AE069460870012006E0802420436C465B
:109440006070C809A0700320694600F0A3FA38BD17
:1094500010B5144603460A4621461120FFF7DCFFEB
:1094600010BD10B50346052200211520FFF7D4FFDB
:1094700010BD10B501210620FFF7B4FF10BDF8B5EF
:1094800005468020694608706B460122112128207C
:1094900000F050F90A20694608706B46012212213B
:1094A000282000F047F90F20694608706B4601221A
:1094B0001221282000F03EF9002469460C706B460A
:1094C000012221462A2000F035F901206946087062
:1094D00002466B4600212A2000F02CF9012D18D0FD
:1094E0000020FFF779FB6B46022203212A20FFF7B9
:1094F00093FF0120FFF770FB6846057846780470FB
:109500006B46012200212A2000F014F93002284382
:10951000F8BD0120FFF702FD6B46022203212A203D
:10952000FFF77AFFE8E710B5034605220021172070
:10953000FFF772FF10BD38B5054600206946087078
:1095400000F0C4F8FF2401342246002D01D003228C
:10955000120200210D2000F0D3F8002D13D06B462D
:10956000012203210F20FFF757FF6846007800070C
:1095700009D5FFF755FE224600210D2000F0C0F866
:109580000020C04338BD002038BD10B5024601217F
:109590000A2000F0C0F810BD10B5044600211A20C2
:1095A000FFF720FF000D22030005120B02430021EC
:1095B0001A2000F0B0F810BD10B5024602492E2066
:1095C00000F09EF810BD000004180000F8B5054634
:1095D0006B46012203210420FFF71EFF0126114CD8
:1095E0003607002D0DD02A4600210C2000F088F807
:1095F000694608781021084369460870A06930431D
:1096000007E069460878EF21084069460870A069BC
:10961000B0430B46A06101220321042000F08AF828
:10962000F8BD00000801002010B5024600211820F6
:1096300000F066F810BD0000F8B507460025684642
:109640000570B807204C2E4600280ADA80206946AB
:1096500008706B46012200210D2000F06BF80120FC
:109660002073F8076946087821D006210843694627
:1096700008706B46012200210D2000F05BF80321E9
:109680000F20FFF799FE8121C900084219D0402020
:10969000694608706B46012200210D2000F04AF84F
:1096A0000020FFF7A9FD00252673ED4309E0022104
:1096B0000843694608706B46012200210D2000F026
:1096C00039F82846F8BD0000280100201CB56B467B
:1096D000012203210F20FFF79FFE684600784022F9
:1096E000C1091040C9014000814208D001206946EB
:1096F0000871024601AB03210D2000F01BF81CBDD0
:1097000008B56B461A70120A5A7089B280B20222EA
:1097100000F010F808BD38B500236C46E254120A78
:109720005B1C042BFADB89B280B22346042200F0D2
:1097300001F838BD38B58024002909D0C025284358
:109740006D462870C8B27F2907D86870022009E0EA
:10975000204369460870012004E020436870C8096E
:10976000A8700320694600F051F938BD10B51446C1
:10977000012312189B029A4202D90020C04310BD57
:109780000B46821E21460920FFF7D4FF002010BDA2
:1097900010B5054A8905126901430A4300210820D2
:1097A000FFF7B9FF002010BD0801002038B50446BE
:1097B0006B4601220E212B20FFF72EFE6846007813
:1097C000E10640094001C90E0143684601706B463D
:1097D00001220E212B20FFF7ADFF38BD10B500216F
:1097E00042541C06120A22431B0A491C0429F7DBB7
:1097F00010BD000013B501231A4669460248FDF763
:10980000D1FD00981CBD0000D0140020FCF70CFE18
:10981000FEF708FDFDF7EAFE3A493B48002522C065
:1098200005608561C56139490562C1600838FCF78A
:10983000F5FEFDF7C7FEFDF79FFFFDF77BFF052651
:1098400001223607D1033046FCF7D9FDFEF786FB2F
:10985000FCF7F8F8FCF7D0F80721B015FFF7B4FCD7
:10986000FFF7C6FC2A4C0A21A08A01224843A084A3
:10987000170339463046FCF7C2FD2348C822254964
:10988000C430FDF731FD244E2079002837D0207AEE
:10989000002834D0FEF7C6FC257120780F2809D99E
:1098A000012239463046FCF7AAFDFEF731FD0022C1
:1098B000394609E0012251033046FCF7A0FDFEF7CE
:1098C00027FD0022012149033046FCF798FDFDF7F2
:1098D000D9FDA08C002801D0401EA0840F48A18C87
:1098E00000780843D0D10121C9023046FCF782FD3F
:1098F0000028C9D101210846FCF746FFC4E7FDF75F
:10990000C1FDC1E7007C00400C140020FFFF0000F7
:10991000B40000206C0C0020000400502A0000203D
:1099200010B50122920218491848FCF701F91648AF
:10993000174902888A4226D0018004218180FF21B4
:10994000F531C1800A21018100211E224181D243CB
:1099500082810122C2810184018241828182C1828D
:10996000018381834323C3860223038778234387AC
:109970008287C2870246403291801184518491844B
:10998000C18300F02DF810BD340D002000FC00084C
:10999000AA550000F0B58C460025102605210907C0
:1099A0008E620E4C08E067467F5DE760A768FF07A0
:1099B000FCD0E7681F706D1C8542F4DB0020074671
:1099C00006E0E760A568ED07FCD0E5681D54401C83
:1099D0009042F6D38E610020F0BD000000300140BF
:1099E00070B572B60124074DA40221462846FCF743
:1099F00085F8002804D0224603492846FCF722F9BE
:109A000062B670BD00FC0008340D0020F0B50025E2
:109A1000102605279C463F070B46BE620C4C06E00D
:109A2000595DE160A168C907FCD0E1686D1C854201
:109A3000F6DB002007E06146095CE160A168C90728
:109A4000FCD0E168401C9042F5D3BE610020F0BD1F
:109A5000003001400000010203040005405C0000EA
:109A6000A05C0400C06C0800805C0400E03F1E00A5
:109A7000E07D1E0007A9022570889B880A00160059
:109A8000010006000100020087008D002D001A3140
:109A900052001A339A001A351D011A376B003B31F8
:109AA000BE003B335E013B3596023B3700009959BF
:109AB0009959EB518F421E45142E0080EB51F52829
:109AC0003333E13A703DE13AC235852BC235333349
:109AD000C235C235AE47E13A5138A33051380000A3
:109AE0000000000000000102030406070809030447
:109AF00006080C10182030000000000102030400CA
:109B0000209B00080000002008010000588B00087E
:109B1000289C000808010020F0180000688B00084D
:109B200000070400091E08054008260910400856D1
:109B300008054008261D040008BE1D040008BED804
:109B4000BC40100800000000000000000000000001
:109B50000000000000000000000000000000000005
:109B600002000000000000000000000000000000F3
:109B7000000000008C0A000000000000000000004F
:109B800000000000000000000000000000000000D5
:109B900000000000000000000000000000000000C5
:109BA00000000000000000000000000000000000B5
:109BB00000000000000000000000000000000000A5
:109BC00005021400090901020081000000000000E4
:109BD0000100000000010000000000000000000083
:109BE0000000000000000000000000000000000075
:109BF0000000000000000000000000000000C8425B
:109C00000000000000000000000000000000000054
:109C10000000000000000000000000000000000044
:089C200000002000000000001C
:04000005080050C1DE
:00000001FF
